:0A00060000308A0007280000840182
:100010001F30830583161F08C0399F009B010730DE
:1000200083129F0019308316990022309800903077
:100030008312980083168501FF30860083128501A4
:10004000831681130D3083120C1A28288316232857
:1000500099000A300C1E2A2899004F300C1E2E28B9
:1000600099004B300C1E322899003E300C1E362869
:1000700099008C1E39281A08A00020080C1E3E2862
:1000800099002008563C031D55288C1E45281A0847
:10009000A10021080C1E4A2899002108303C0319B0
:1000A00005102108313C031905142008413C031DAB
:1000B00069288C1E59281A08A10021080C1E5E28E8
:1000C00099002108303C031985102108313C03199F
:1000D00085142008523C031D7D288C1E6D281A08AB
:1000E000A10021080C1E722899002108303C031938
:1000F00005112108313C031905150D300C1E7E2811
:0E01000099000A300C1E822899002D286300F9
:040000008A01032846
:02400E00693F08
:00000001FF
